S10E24008E0FFFBD27D54FCE20008CAF
S111240B200C2705A7000820F6CE27DC18CEEB
S111241920008C27DC270AE60018E7000818CC
S11124270820F1CC0000270CC3200C3736CC63
S10E2435200CBD279038BD244020FE81
S1112440BD272B04C63FF710097F2009C6FFF5
S110244EF72008CC003CBD24AECC000CBD32
S111245B24AECC0006BD24AECC0001BD24AEE0
S1102469CC0080BD24AECC2707BD24E9CCF7
S111247600C0BD24AECC26FCBD24E9CC0094ED
S1102484BD24AEBD25BEED026D0327F7F6A5
S111249120094F5D2A0143BD24CB20EA8FC3EE
S111249F00048F353839F6B5F0C4805D26F898
S11024AD3937363C3C30EF00EC04E705BD48
S11124BA24A5E605F7B5F08FC300028F353870
S11124C818383937363C3C30EF00BD24A5E609
S11124D6054F5D2A0143F7B5F18FC300028F55
S11124E4353818383937363C3C30EF002015B7
S11124F21AEE0418E6004F5D2A0143BD24CB08
S1112500EC04C30001ED041AEE04186D00266D
S111250EE38FC300028F3538183839BD272BF0
S110251C46EC08272BCC0000ED02201DCC5E
S11125290000ED042007EC04C30001ED04ECF7
S1112537041A83004925F1EC02C30001ED02F1
S1112545EC021AA30823DC8FC300068F35387E
S1112553183839BD272B46EC082731CC000080
S1112561ED022023CC0000ED04200DCC00017F
S111256FBD2519EC04C30001ED04EC041A832D
S111257D006425EBEC02C30001ED02EC021A2F
S111258BA30823D68FC300068F3538183839BD
S1102599C68BF7B5F7C6FFF7B5F4C693F788
S10B25A6B5F7C6FFF7B5F639DD
S11125AE4423302A433938374236353441331A
S10525BC3231B6
S11125BEBD272B14EC00C3000418CE25AE3C40
S11125CC8FCC0010BD271338BD2599CC000A12
S11125DABD2519C60FF7B5F6F6B5F4F72007C0
S11125E8C8FF5D2610C6FFF72008CC00008F48
S11125F6C300148F353839F62008C1FF270BB7
S1112604CC00008FC300148F3538397F2003BB
S1112612C680F720062036F620064F8800C842
S1112620FFF72005F7B5F6F6B5F4F720044FE2
S111262E8800C8FFF720047D20042702201A2C
S111263CF620034FC30004F72003F620064FD8
S110264A4756F72006F62006C10F22C37D77
S11126572004260BCC00008FC300148F3538EE
S110266539F6B5F4F72007C680F72006F615
S11126722007F420065D2626BD2599EC00C342
S11126800004ED02F620034FE302188F18E663
S111268E00F72009F72008CC00018FC30014C8
S111269C8F353839F620034FC30001F72003B1
S11126AAF620064F4756F72006C10826BABD93
S11126B82599CC00008FC300148F3538398F5C
S11026C6C300148F353839CC00003939BDFC
S11126D3272B042003BD26CDBD25BEED026DD0
S11026E10327F4F620094F5D2A01438FC33F
S11126EE00048F3538398FC300048F35383916
S11126FC5072657373204B657973004B6579DA
S10C270A706164205465737400CD
S11127131A83000027113718E600E70033830D
S10D27210001270508180820EF390D
S111272B1838181F00400237363C3018E600FC
S11127394FC43F37368F30A3008F35EF0018A2
S11127471F0080043C3C3C3C186E01183037E7
S111275536188FC30001183018EE0218EB007E
S11127638900188F3233183C183018AE001855
S1082771EE02186E01E8
S111277637363C303C30EC04F7102BC60CF721
S10F2784102D8FC300028F35381838392F
S1112790BD272B46EC08ED041AEE04FC200ACB
S111279E18ED00EC04FD200AEC08C30006ED63
S11127AC02EC0CA3023736EC04C30004188FB1
S11127BA323318ED00EC04C30002188FEC0C4F
S11027C818ED008FC300068F35381838391E
S10A27D5CC0030BD2776396A
S9032400D8
